:020000040000FA
:020000001328C3
:08000800A0000308A10021087B
:100010008300A00E200E090007308A002208003E4F
:1000200003188A0A8200462052207B203A20412071
:10003000A801AE0A0319AD0A03194120061C1828AD
:10004000A80A031918280000000000000000061884
:100050002028A1203A20C1306320290861202E30B9
:1000600061202A0861202B0861206D3061207330E7
:100070006120182880306320003073200F307320F7
:100080000800C13063201630732008000B12850170
:1000900007309F0083160313F83085000130860077
:1000A000831208008D2030306320383063200E30FA
:1000B00063205D20253073200800013063208D20EF
:1000C00008000314642803100515A3000930A400D8
:1000D0000514031C0510851000008514A30CA40B47
:1000E000682805110800A2000C20003A0319080036
:1000F0006120A20A7428803063201D3073200030F4
:100100007320C030632006307320972097209720FB
:100110009720972097205D2008009F30A500103081
:10012000A600A50B9428A60B9128962808004F300E
:10013000A500C430A600A50B9E28A60B9B28A028CE
:1001400008000830AC00A901AA01AB010530290262
:100150000318CA2005302A020318CD2005302B02CF
:100160000318D020AC030310A80DAB0D2B1AD3201D
:10017000AA0D2A1AD620A90D03102C08031DA628A3
:100180002908303EA9002A08303EAA002B08303E3C
:10019000AB0008000330A90708000330AA070800D5
:1001A0000330AB0708002B12031408002A120314B3
:0201B000080045
:100E0000503455344C3453344534003443344F3427
:100E100055344E3454342034563431340034203474
:100E20006934733400346D347334003430342E3408
:100E3000303430346D34733400345234433420341D
:0C0E40000034203400342034003400342E
:02400E00A13FD0
:00000001FF
